:020000040000FA
:10000000502D0020F902000001030000030300004E
:1000100005030000070300000903000000000000C2
:100020000000000000000000000000000B030000C2
:100030000D030000000000000F030000110300008A
:100040001303000021070000E10A00001303000071
:1000500013030000130300007D04000013030000DD
:100060007D0A0000130300001303000013030000C7
:100070001303000013030000130300001303000028
:1000800013030000B1070000130300001303000076
:10009000D5070000D9070000130300001303000078
:1000A00013030000130300001303000013030000F8
:1000B0001303000013030000000000000000000014
:1000C00013030000130300001303000013030000D8
:1000D00013030000130300001303000013030000C8
:1000E00013030000130300001303000000000000CE
:1000F00000000000130300000000000013030000D4
:1001000000000000000000000000000000000000EF
:1001100000000000000000000000000000000000DF
:1001200000000000000000000000000000000000CF
:1001300000000000000000000000000000000000BF
:1001400000000000000000000000000000000000AF
:10015000000000000000000000000000000000009F
:10016000000000000000000000000000000000008F
:10017000000000000000000000000000000000007F
:10018000000000000000000000000000000000006F
:10019000000000000000000000000000000000005F
:1001A000000000000000000000000000000000004F
:1001B000000000000000000000000000000000003F
:1001C000000000000000000000000000000000002F
:1001D000000000000000000000000000000000001F
:1001E000000000000000000000000000000000000F
:1001F00000000000000000000000000000000000FF
:10020000DFF80CD000F00AF900480047B1190000EF
:10021000502D002030B4044654E8000F0D4644E849
:100220000053002BF8D1156030BC704730B4044641
:1002300054E8000F40EA010544E80053002BF7D1D1
:10024000156030BC704730B4044654E8000F00EA33
:10025000010544E80053002BF7D1156030BC70470E
:1002600030B4044654E8000F80EA010544E8005326
:10027000002BF7D1156030BC704730B4044654E809
:10028000000F00EB010544E80053002BF7D1156087
:1002900030BC704730B4044654E8000FA0EB0105B1
:1002A00044E80053002BF7D1156030BC704770B4A0
:1002B00004464FF0000054E8006F0D68AE4207BFDF
:1002C00044E80023012044E800630E60002B1CBFBB
:1002D0000020F0E770BC704730B4044654E8000FCB
:1002E00088422CBF451A054644E80053002BF5D13F
:1002F000156030BC7047000006488047064800473C
:10030000FEE7FEE7FEE7FEE7FEE7FEE7FEE7FEE7C5
:10031000FEE7FEE74D080000010200002DE9F05F56
:100320000546002092469B46884606468146402464
:100330001BE0284641464746224600F05EF85346F9
:100340005A46C01A914110D311461846224600F071
:1003500016F82D1A67EB01084F46224601200021AE
:1003600000F00DF817EB00094E41201EA4F1010426
:10037000DFDC484631462A464346BDE8F09F202A46
:1003800004DB203A00FA02F1002070479140C2F1EC
:10039000200320FA03F31943904070470048704748
:1003A0005864000040EA01039B0703D009E008C934
:1003B000121F08C0042AFAD203E011F8013B00F82A
:1003C000013B521EF9D27047D2B201E000F8012B76
:1003D000491EFBD270470022F6E710B513460A46C5
:1003E00004461946FFF7F0FF204610BD421C10F8E6
:1003F000011B0029FBD1801A7047202A04DB203A18
:1004000021FA02F00021704721FA02F3D040C2F134
:10041000200291400843194670470000064C074DE2
:1004200006E0E06840F0010394E8070098471034C4
:10043000AC42F6D3FFF7E8FE3C6500005C650000C7
:1004400030B58C1810F8012B12F00F0301D110F801
:10045000013B120906D110F8012B03E010F8015BF3
:1004600001F8015B5B1EF9D101E001F8013B521E6E
:10047000FBD1A142E6D3002030BD00002DE9F04FB2
:1004800000268DB0DFF8A081B14604964FF4807548
:10049000012437460596284602F0EEF938B1D8F81F
:1004A0000403204203D0284602F0DCF926432D1D28
:1004B00064007F1CADB2082FEDD34FF4BE7420460C
:1004C00002F0DAF948B1204602F0CCF946F00046D5
:1004D00004AA0221002002F0AFF9544C16F0FF0FDD
:1004E00015D00127002537420DD008EB8501D1F842
:1004F0001005D1F81015C0F3052054F82520C1F3DC
:10050000014102B190477F006D1C082DEBD3002EF6
:100510007EDA0020CDF82890411E0DF1100B07AABD
:10052000CDF82C9042F82010401C91460228F9D3B7
:1005300000252E46A11911F8607F91F9000027F0DF
:10054000C008401C40D007A9404601F08BFC40B3D6
:100550004FEA971A404600F051FF54F820701FB13F
:10056000BAF1030F03D006E0BAF1030F2CD10AA9A8
:10057000404601F07FFC02A8CDF8088002F000F9A7
:10058000029900EB8100D0F8000704A9C0F30140F4
:100590000290404601F066FC0028029802D0022832
:1005A00002D011E003280FD1BAF1030F08D102984D
:1005B000022833D00221404602F0BCF86D1CEDB297
:1005C00017B151464046B847761C042EB2D3002DD1
:1005D00021D001AA0221002002F02EF900205A4663
:1005E0000DF1040152F8206051F82030B34217D0C9
:1005F00000200AAE4FEA090351F8207042F820703B
:1006000056F8207043F82070401C0228F4D300E014
:1006100001E0002D8CD10DB0BDE8F08F0321CAE7B9
:10062000401C0228DED3F6E7006000407C02002078
:1006300000F01F02012191404009800000F1E020FC
:10064000C0F88012704700F01F020121914040095C
:10065000800000F1E020C0F88012704700F01F0217
:10066000012191404009800000F1E020C0F8801293
:10067000704700F01F02012191404009800000F105
:10068000E020C0F88012704700F01F020121914065
:100690004009800000F1E020C0F88011704700F0B0
:1006A0001F02012191404009800000F1E020C0F8C4
:1006B0000011704700F01F020121914040098000A5
:1006C00000F1E020C0F80011704700F01F02012186
:1006D00091404009800000F1E020C0F8001270470E
:1006E0004907090E002806DA00F00F0000F1E020AB
:1006F00080F8141D704700F1E02080F80014704766
:100700004907090E002806DA00F00F0000F1E0208A
:1007100080F8141D704700F1E02080F80014704745
:1007200070B5204D28696C78401C2861687D10B137
:100730001D4801F027FB287803281AD11B48D0F860
:100740000C01B0B1012C04D0022C0AD01648123092
:1007500023E02869032816D01348083001F012FB63
:1007600011E02869022812D00F480D3001F00AFB71
:100770000DE0032C0FD2012C05D0022C07D0BDE8D0
:10078000704003F095BABDE8704003F0BDBABDE813
:10079000704003F0CFBC04482830BDE8704001F041
:1007A000F1BA0000040A002038030A0000100040DB
:1007B00007480021C0F84011C0F84411C0F84811A2
:1007C000C0F84C11C0F80011C0F8041105F028BBA6
:1007D0000010014005F076BA30B51B4C85B00025FD
:1007E000012080F31088D4F8D40038B3D4F8D000B6
:1007F00000EB800004EB800001798DF80010816827
:10080000C26803694069CDE90330CDE90112D4F82B
:10081000D400401EC4F8D400D4F8D000401CC4F862
:10082000D000D4F8D0000A2801D3C4F8D05000205A
:1008300080F31088216868468847D1E7002080F35C
:10084000108805B030BD0000200A002030B54FF000
:10085000805000228300D0F83011C3F80C21C3F877
:100860001021624B1A60624B1B68624C2360604B24
:100870001B1D1B68241D23605D4B08331B68241D52
:1008800023605B4B0C331B68241D2360584B1033D3
:100890001B68241D2360564B14331B68241D2360E2
:1008A000534B18331B68534C20342360504B1C337C
:1008B0001B68241D23604E4B20331B68241D2360BE
:1008C0004B4B24331B68241D2360494B28331B6882
:1008D000241D2360464B2C331B68241D2360444B8E
:1008E00030331B68434C40342360414B34331B6826
:1008F000241D23603E4B38331B68241D23603C4B72
:100900003C331B68241D2360394B40331B68241D76
:1009100023600124082902D1D0F8343113B1082909
:1009200004D006E0354B3449196005E0D0F8343185
:1009300013B1082904D006E0314BFB21196005E012
:10094000D0F8343113B1082908D00EE090F85832AD
:100950002C48016863F30301016002E0D0F83431F0
:100960001BB929494FF40070086028480168C9077D
:1009700002D06FF0010101602548016841F4700167
:100980000160BFF34F8FBFF36F8F4FF01021D1F88D
:100990000002002803DBD1F80402002822DA1D4BF4
:1009A0001C601D480468002CFCD01224C1F80042D1
:1009B0000568002DFCD0C1F8044201680029FCD074
:1009C0001A6001680029FCD0BFF34F8F10487C38B3
:1009D0000168124A01F4E06111430160BFF34F8FD7
:1009E00000BFFDE70F490E48086030BD38050040E4
:1009F0000404001020C50040488103008C560040CC
:100A000018F50040E40E004040960240000400400B
:100A100088ED00E004E5014000E401400400FA052F
:100A20000090D003DC000020124A10B50021104BCA
:100A3000126809E053F82140844203D10E4801F0C6
:100A4000A1F913E0491CC9B29142F3D3084A00212D
:100A500012F1180201EB011302EB4303834201D1AF
:100A6000012010BD491CC9B20629F3D3002010BDD6
:100A70006C0C00204C010020EC00030070B5144EFB
:100A80004FF48030C6F808030025C6F84051114CD9
:100A9000606810B9104801F075F9A570626801230B
:100AA000656073640D480168001F00681430B1F57B
:100AB000804F04D2B0F5404F01D9637005E0814208
:100AC00001D3012000E000206070BDE870401047B5
:100AD0000080004024010020E5000400448500401F
:100AE00001480068004700002800002002E008C814
:100AF000121F08C1002AFAD170477047002001E098
:100B000001C1121F002AFBD17047022000F0EEB98C
:100B100070B50024064D06E06868012110F8340025
:100B200004F008FC641C28788442F5D3002070BDD2
:100B300030000020F8B515460C460646052A01D2BD
:100B40000720F8BD04F0EEFC18B904F0B1FC002851
:100B5000F7D1124900224E600C708D60C1E9042269
:100B6000C1E906220E4D0DE006EBC4002968009194
:100B700081788DF8011000780A4A694604F026FC55
:100B80000028DED1641EE4B2EED2BDE8F84004488D
:100B90000021054A001D00F053B80000300000207D
:100BA00054630000A5150000B914000072B604F0EB
:100BB00059F800BF03F09CFE0028FBD1104C012126
:100BC000208801EB00400FA103F09EFF1048006851
:100BD000C00700D000BE2088022101EB00400DA11B
:100BE00003F092FFBFF34F8F0948E43801680D4AC4
:100BF00001F4E06111430160BFF34F8F00BFFDE7D7
:100C000064010020466174616C206572726F72002D
:100C1000F0ED00E053797374656D2072657365744F
:100C2000000000000400FA050EB500210091CDE996
:100C300001106A4644F20100FFF7B8FF0EBD000044
:100C4000074B9B7823B12AB120B10068037C1BB10C
:100C500008207047072070474174426100207047A8
:100C60005803002070B504F079FF104800240B21D0
:100C7000047044700E4D817014206C602C706C7088
:100C8000FFF7D6FC07211420FFF72AFD1420FFF7F9
:100C900006FD0848046007211120FFF721FD0548E3
:100CA000001F0068A860002070BD000058030020ED
:100CB00050000020081501402DE9F843DFF870903E
:100CC00099F802305BB350B3052902D20720BDE882
:100CD000F88343691BB3437C012B22D000270446D1
:100CE000002588461646284600F036F8684605F086
:100CF000F7FAC0B1012101700E4944600968C0E9EA
:100D00000218C0E904769DF8000089F8010000206F
:100D100000F024F81420FFF7D8FC2846D7E7082075
:100D2000D5E70F46DBE70425002000F017F8F4E7CD
:100D300058030020041501400649897839B130B1C3
:100D4000416921B100210174022105F049B8082050
:100D5000704700005803002000F002B800F008B807
:100D600072B602480168491C0160704764000020A7
:100D700003490868401E086000D162B67047000051
:100D80006400002070B5054608680C46411C04D07C
:100D900001F02BFD206801F0B9FC6068411C02D015
:100DA000002101F0A1FC2968A069C1F82405607D3B
:100DB000227D29681043C1F86C05D4E90012286827
:100DC000C0F81425C0F80C15207D012814D1A068A6
:100DD000411C02D0002101F087FCE068411C04D0D6
:100DE00001F003FDE06801F091FCD4E902122868EB
:100DF000C0F80825C0F8101570BD70B50546086824
:100E00000C46411C04D001F0FAFC206801F088FC7B
:100E10006068411C02D0002101F06FFC2968A069C4
:100E2000C1F82405607D217D2A680843C2F86C055D
:100E3000D4E900122868C0F80C15C0F81425207DEC
:100E4000012814D1A068411C02D0002101F055FCFA
:100E5000E068411C04D001F0D2FCE06801F060FCC5
:100E6000D4E902122868C0F80825C0F8101570BD32
:100E7000084908B5085C0090684601F073FCD0F89A
:100E800010050099C84010F0010000D0012080F04A
:100E9000010008BD146300002DE9FC410646C007AF
:100EA0004FF000050ED0104F00240122385D009550
:100EB00000231146019501F0A1FB641C042CF4D31E
:100EC00000F04EF8B0070DD5074E0024361D002265
:100ED000305D032300951146019501F08FFB641CE2
:100EE000042CF4D3BDE8FC8110630000094908B567
:100EF000085C0090684601F035FCD0F80425009BA2
:100F00000121994021EA0203C0F808351140C0F8D8
:100F10000C1508BD106300000249085C012101F0B6
:100F200078BC0000106300000249085C002101F059
:100F300070BC000010630000084908B5085C009010
:100F4000684601F00FFCD0F804050099C84010F085
:100F5000010000D0012080F0010008BD10630000F6
:100F600010B500242046FFF7D7FF641C042CF9D3EA
:100F700010BD10B500242046FFF7D6FF641C042CDA
:100F8000F9D310BD10B50246064B4FF0FF300021DB
:100F90005C5C944201D1084610BD491C0429F7D37A
:100FA00010BD0000146300002DE9F0470D46814696
:100FB000FFF7E8FF0446042836D2DFF874801B48A8
:100FC0001C4EA8F10C0725B3012D0ED0022D2BD1FC
:100FD00004EB440030444578002D25D0B968002941
:100FE00022D02846BDE8F047084704EB4401755C71
:100FF0000E44717849B10E4A4FF40041093A8068B5
:10100000FFF75AFE08B987F80390B17808F8041082
:10101000E2E78068FFF790FE04EB4401314418F8E2
:1010200004008D78A842D7D0BDE8F087186300008F
:101030001000002050020020042801D2FFF718BF42
:101040000020704770B50023042810D20D4D00EB2E
:101050004004012A02D101290CD00022094E00EBE4
:101060004000304461B1012906D0022906D007238F
:10107000184670BD0E30C2B22A55F9E74270F7E744
:101080008270F5E75002002070B506461E48002425
:10109000C0E90161B00720D500250122114628468C
:1010A000FFF7D0FF6D1C0446042D02D2002CF4D0B3
:1010B00013E094B940F2666204211448FFF73AFD48
:1010C00004000AD1FFF724FD040006D10F48104A9E
:1010D0000021001FFFF7B4FD0446F00712D00120E5
:1010E000FFF7DAFE74B909480A4A00210C38FFF705
:1010F000A7FD040006D10548074A01210838FFF77B
:101100009FFD0446204670BD0400002024630000BB
:1011100091130000091800000B0B00002DE9F05F8F
:101120006A4C054600266078B34618B184F801B0D1
:1011300000F052FB664F4FF47A694FF4C87A4FF0D3
:101140000108182D62D2DFE805F0AC0C0C31404DDF
:1011500062676B746B74BE7D7D7D7D7DACAFB2B517
:10116000BEBE0020FFF7E8FE00284FF0000008D0C8
:10117000FFF7D2FE022D02D14FF4E16008E04846AD
:1011800006E0FFF7D1FE022D01D1C82000E0504655
:10119000410CC0034FF4FA72801841F10001257030
:1011A00052000023FFF7BAF801462AE00020FFF7BB
:1011B000C3FE00284FF0000004D0FFF7ADFE4FF44F
:1011C0004870E5E7FFF7B0FEDFE70020FFF7B4FE69
:1011D00000284FF0000002D0FFF79EFECFE7FFF798
:1011E000A3FED4E70020FFF7A7FE00284FF0000081
:1011F00002D0FFF791FE01E0FFF796FE257041F661
:101200009A1100223868FFF757FD064646E0002095
:10121000FFF76CFE257008E0002051E025703DE0EE
:1012200084F801800120FFF761FE002240F6CD41E5
:10123000E8E784F801800120FFF758FE00224FF410
:101240008041DFE77868FFF777FD0646D5F11100AA
:1012500000D02EB10220FFF75FFE84F802B01DE03F
:10126000012816D980B2C8214843C117C90341EAF1
:101270005041C0034FF4FA72801841F1000152004E
:101280000023FFF74BF8014600227868FFF714FDB2
:1012900006460220FFF748FE84F802803046BDE88B
:1012A000F09F00F099FAB9E700F096FAB4E700F081
:1012B00093FA04E000F090FA0020FFF735FE0120D9
:1012C000FFF732FEAAE7FFF754FEA7E7040000206D
:1012D000186300002DE9F0470546861C90460F462E
:1012E0004FF001090020FFF737FD1B4C20683860E4
:1012F000D4E90001401AA16804F21C47081A0EE064
:101300000121384600F046FD00F004FB0146384656
:1013100000F040FDD4E90001401AA168081A401C01
:101320008642EDD8B8F1000F03D0052065F389108F
:1013300002E0062065F39F50A2682168114004EB8B
:101340008101C8602068304420600020FFF706FD5E
:101350004846BDE8F08700006405002030B482688C
:101360000468531C8360A154D0E901128A4202D35D
:1013700030BC01F04AB830BC70470000034803C8D5
:10138000814201D101207047002070476405002090
:1013900000780221FFF708BE05494FF0FF32082808
:1013A00041F8202002D3084480F8582070470000FC
:1013B0007C020020F0B54FF0FF3512B10023082663
:1013C00001E008230C260C4C05E000BF54F8237004
:1013D0007F1C04D05B1CB342F8D32846F0BD26180E
:1013E0005DB286F8305044F82310002AF5D1E11898
:1013F00081F85800F1E700007C020020024908440F
:1014000090F93000704700007C0200202DE9F05F69
:1014100026484168F1B3DFF898B00E688146DBF8E2
:10142000004087688078E11B21F07F45ED1CB0B952
:10143000DFF880804FF48030C8F84403C8F8040314
:101440001120FFF7F5F81120FFF729F94FF0010AF5
:10145000C8F800A02F2003F065FF89F802A0B5426C
:1014600000D23546124BE8193C3320F07F4018601B
:10147000DBF800105A46091B21F07F41001B20F0C9
:101480007F40C91C81420FD9106818602F2003F0DB
:1014900049FF00E004E0BDE8F05F1120FFF715B957
:1014A000BDE8F05F04F05ABBBDE8F09F500000209B
:1014B00004150140001001402DE9F0470025DFF838
:1014C0008C803CE06068002100EBC506012032788A
:1014D0009146FEF754FFD4E9062300EA020701EA29
:1014E000030C57EA0C0728D082438B434846C4E9D3
:1014F000062303F0D5FF3278824691460120002171
:10150000FEF73DFFD4E9042300EA020401EA0307E1
:101510004A4650460021FEF732FF44404F403C43CC
:101520000BD17078012801D0012100E00021726800
:1015300081EA0A010AB1484690476D1CEDB298F85D
:10154000000044468542BDD3BDE8F087300000204E
:1015500010B50021024800F028FC80F3100010BDF7
:10156000800900200E4910B50A784C780023A24269
:1015700012D0521CD2B20A70022A00D10B70084A53
:101580000B780C3252F8232002608868104420F057
:101590007F408860012010BD0360002010BD000066
:1015A000500000202DE9F041804602460120002134
:1015B000FEF7E5FE1A4F05460E467868FFF7BCFBBE
:1015C00000280CD1174CD4E9062110462A4001EA24
:1015D00006031A4305D0A843B143C4E90601BDE898
:1015E000F081404603F05CFF30B1D4E904012843A8
:1015F0003143C4E9040105E0D4E90410A943B04330
:10160000C4E90410D4E9060128433143C4E90601C2
:10161000A1687868BDE8F0410022FFF74DBB0000EB
:1016200054630000300000200278521C02700278DF
:101630008A4201D30021017070472DE9F041002555
:101640002C4601272046FFF7F7FC18B107FA04F6ED
:101650002E43F5B2641C042CF4D3E843C0B2BDE8B9
:10166000F08100002DE9FC5F0E008346DDE90C47A8
:10167000C6F1000098469246814600D408460125EE
:1016800003E000BF90FBFAF06D1C5045FADAA84564
:1016900000D9454624B1002E01DB780700D5641E31
:1016A000B80702D5B8F1000F0AD0F80708D13CB14D
:1016B000A54205D220215846641EFFF74FFEF6E7EB
:1016C000002E02DA4E462D2102E0780703D52B21A9
:1016D0005846FFF743FE07F0030002280BD1B8F18C
:1016E000000F08D13CB1A54205D230215846641EF6
:1016F000FFF734FEF6E7CDE9004743465246314650
:10170000584604F093FDBDE8FC9F000070B50D46FF
:10171000044600684FF4887103F0FEFD4FF49071A9
:10172000206803F0F9FD4FF49271206803F0F4FD96
:101730004FF4A271206803F0EFFD20681249C0F851
:10174000041320686907000B40B2090E002806DA6E
:1017500000F00F0000F1E02080F8141D03E000F11C
:10176000E02080F8001420680121000B40B200F056
:101770001F0291404009800000F1E020C0F8801273
:10178000C0F8001170BD00001003020002460020E6
:101790001268930702D0530702D47047500714D53C
:1017A00002F00300012802D002280CD105E0C2F3A8
:1017B00083100B68801C184404E00223086803EBC4
:1017C00092521044086001207047086800EB925361
:1017D000C2F38910401CEEE70A4810B5807860B16A
:1017E000002401E0022C06D02046FFF795FB641C84
:1017F000042CF7D310BD0324F6E7BDE81040FFF733
:10180000AFBB00000400002003480179C90702D0E3
:101810000078FFF783BC7047040000202DE9F047F3
:10182000394E002780463D46DFF8E090D6F804A008
:1018300057E003D00446D0F81C8035E099F800202A
:1018400002EB4201521CD2B289F8002009EBC1011F
:1018500099F80230091D9A4201D189F80050486870
:101860000A780446012A12D0022A02D0032A3BD168
:1018700008E004F085FA00B10127257434E005740E
:10188000C06900E070680028F9D170602CE0207C0D
:1018900050BB88686060C868A0600869E0604869FB
:1018A000A061F07800B165606268B168184B501AA9
:1018B00020F07F40984202D2A168084406E0881ACE
:1018C000A16820F07F40814202D9081A206000E020
:1018D000256065600120A56020742046E56104F064
:1018E00031FAB8F10000A4D199F8001099F801007C
:1018F0008142A3D117B97168514502D00120BDE8DA
:10190000F0870020FBE70000500000205803002073
:10191000FFFF7F002DE9FF410026234800F037FA42
:101920002148001F074600F032FA204C6068009002
:10193000A56800E000986946284004EB80000C3060
:10194000FFF724FF0028F5D101AA009901EA050359
:1019500004EB8303491CDB6842F82030401C0091F3
:101960000228F2D3019800F0030001280BD00228CE
:1019700010D10198032101EB90500099BDF80A6045
:1019800001EB900005E00198BDF80A60C0F38310F8
:1019900008440090384600F0F7F908B100986060FC
:1019A00004B03046BDE8F0817C09002064050020C9
:1019B00008B504F0F9FB002001F0A4F828B901F003
:1019C00099F800F50340FFF72FF9642001F04CF976
:1019D000364801F09BF928B901F08CF800F5034076
:1019E000FFF722F9FFF729FE314901220870002094
:1019F00000F04AFF2F4E58B93088012101EB00401A
:101A00002DA103F081F800BF02F072FF0028FBD186
:101A100001F01AF828B901F06DF800F50340FFF75E
:101A200003F93088032505EB004027A103F06CF88B
:101A30001E4C00BF02F05CFF0028FBD120BF2068D5
:101A4000B0F57A7FF6D30020FFF786F930880521BC
:101A500001EB004027A103F057F8308826A105EBE1
:101A60000040226803F054F830882CA105EB0040B8
:101A7000626803F04DF800270EE000BF04EB87001A
:101A80003A4681680091836C30882E4905EB00400E
:101A900003F045F87F1CFFB201F026F8B842EDD8FC
:101AA0000020FFF75BF901F073F8C3E7880100201D
:101AB00000000020640100205458206669666F20F1
:101AC0006572726F72200000477A6C6C2061636BE4
:101AD000207061796C6F616420646576696365204C
:101AE0006578616D706C6520737461727465642EC5
:101AF000000000000D0A0000546F74616C207472C5
:101B0000616E736D6974746564207061636B657474
:101B1000733A20202025347500000000546F746152
:101B20006C207472616E736D697373696F6E20746B
:101B3000696D652D6F7574733A20253033750D0A04
:101B4000000000005C6400002DE9F047C7880446EF
:101B5000181D16468946B0FBF7F1B0FBF7F207FBFC
:101B600012009A193A44D21CB2FBF7F2DDF820A019
:101B700001E02468491E0029FBD13D1A8846B54280
:101B800016D818E0BAF1000F05D0211809EB0800AB
:101B90002A46091D04E0204409EB08012A46001DDD
:101BA000FEF700FC00202468761BA844B74201D948
:101BB000354600E03D46002EE4D1BDE8F087000048
:101BC00030B5024659B103F035F80021074C09E061
:101BD00004EB810315685B88AB4202D111600020E1
:101BE00030BD491C8142F3D3052030BD5001002097
:101BF0002DE9F0415C4903780446D1E90302002550
:101C0000082B77D2DFE803F0042B4877726E8795B4
:101C1000217C914208D238B100EB81018A6C521CC0
:101C20008A640168491C0160A17B2E4661F30706A6
:101C30002189677B61F31F466189606861F30F0545
:101C4000217B61F31745E17B61F31F6501F07EFCA9
:101C50002A4631463846BDE8F04100F095BE486955
:101C6000407D10B9414800F08DF82F46218965F379
:101C7000070761F31F476189267B61F30F05617BCD
:101C8000606861F31F6501F061FC2A463946304601
:101C9000BDE8F04100F040BE217B914208D238B14E
:101CA00000EB81018A6C521C8A640168491C016046
:101CB000A07A217A60F3070561F30F25E17A667A4D
:101CC000676861F3174538B11FB92848263000F01E
:101CD00059F8384601F03AFC29463046BDE8F04153
:101CE00000F00EBFBDE8F04100F0ACBE00F04EFFCA
:101CF000BDE8F08131E01E484168491C416001782F
:101D00000029F5D0816811B1491E8160F0E7BDE876
:101D1000F04100F08BBEA379934208D238B100EBBA
:101D2000830293685B1C93604268521C42608A681D
:101D30000CE0A379934208D238B100EB8302936898
:101D40005B1C93604268521C42604A68002ACFD0F4
:101D500061792079BDE8F0411047BDE8F0410348C2
:101D60007F3000F00FB80000E00000203D040500C7
:101D70008809002002490F220A708861704700001C
:101D8000E0000020FFF7F6BF002100F009B80121B4
:101D900000F010B808B56A46FEF76FFA009808BD63
:101DA00008B56A46FEF74FFA08BD08B56A46FEF761
:101DB00031FA08BD08B56A46FEF738FA009808BD42
:101DC00008B56A46FEF766FA009808BD70B5044685
:101DD00000252846FEF7C0FF216862680868904227
:101DE0000ED9401E08600178A38AE26801FB032532
:101DF000227A2168101AC0B20A79824200D2087190
:101E00000020FEF7ABFF284670BD70B505460C46B6
:101E10000020FEF7A1FFE868A98A201AB0FBF1F1C3
:101E20002A681068431C13600170BDE870400020F0
:101E3000FEF794BF10B530B1017A42680368891A81
:101E4000C9B21A6006E00E2010BD03681A68541C5F
:101E50001C601170491EC9B2F7D2006800210171DF
:101E6000084610BDC20800F007030120895C9840B5
:101E70000840704710B5C20800F00703885C0124D1
:101E80009C402043885410BD70B5074C251F206826
:101E900029684968884202D30448FFF773FF28681D
:101EA00021688068405C70BD1C0100204400010076
:101EB00001480068704700001C01002010B504466E
:101EC000054800684068A04202D80448FFF75AFF5E
:101ED0000148001D046010BD180100204C000100E5
:101EE00001484068704700001C01002010B50446FE
:101EF000054800680068A04202D80448FFF742FF86
:101F00000148001D446010BD180100205800010068
:101F100010B5040002D10548FFF734FF0448002142
:101F20000460001D0160416010BD00002700010039
:101F3000180100200948021F4168491C41601268CD
:101F40001368994208D3002343600168491C01606B
:101F50005268914200D30360704700001C010020CA
:101F6000002839D0401E00BF00BF00BF00BF00BF27
:101F700000BF00BF00BF00BF00BF00BF00BF00BF69
:101F800000BF00BF00BF00BF00BF00BF00BF00BF59
:101F900000BF00BF00BF00BF00BF00BF00BF00BF49
:101FA00000BF00BF00BF00BF00BF00BF00BF00BF39
:101FB00000BF00BF00BF00BF00BF00BF00BF00BF29
:101FC00000BF00BF00BF00BF00BF00BF00BF00BF19
:101FD00000BF00BF00BFC5D170470000F0B5054687
:101FE0000478154889B0164640F82420124A08693A
:101FF0000832A2F10C0742F82400487F385520220D
:102000006846FEF7CFF904942878385C48B10EB1E1
:102010000A4A00E000226946281D03F0EDFB09B0E2
:10202000F0BD0EB1064A00E00022694605F10C0041
:1020300003F0B4FAF3E70000180000208560000008
:10204000D15E000001480068704700004C0100208C
:1020500010B50020114A014600EB40039C18617046
:10206000A170D154401CC0B21028F5D3DE22CC217F
:102070000B48FEF7A9F90A4A0020A2F1180100BF97
:1020800000EB001302EB430341F82030401CC0B2C8
:102090000628F5D303490620086010BD7C0B0020FC
:1020A000840C00204C01002070B5104C06462068BE
:1020B000062802D30E48FFF765FE3046FEF7B4FC53
:1020C00018B90B48401CFFF75DFE0A4D20680A490D
:1020D00055F82000884203D00548801CFFF752FEC7
:1020E000216845F82160491C216070BD4C01002029
:1020F000800003006C0C0020ADDEADDE10B50446A0
:10210000102802D30348FFF73DFE034904EB4400C7
:10211000085C10BDC20003007C0B002070B50026D7
:102120000446102802D30C48FFF72CFE0B4D04EB9D
:102130004404285D70B105F1300000EB84016019A2
:1021400010F8022F51F822600321FFF76DFA285D85
:10215000401E2855304670BDA20003007C0B0020B5
:1021600070B50C460646102902D31248FFF70AFE46
:102170003046FEF759FC18B90E48401CFFF702FE26
:102180000D4D04EB4404285D032810D205F1300006
:1021900000EB8401601910F8012F41F8226003213F
:1021A000FFF742FA285D401C2855012070BD002031
:1021B00070BD00008C0003007C0B002010B50446AD
:1021C000102802D30948FFF7DDFD094904EB44005C
:1021D0000A5C42B101F1300202EB800208448078CF
:1021E00052F8200010BD002010BD0000B300030015
:1021F0007C0B00200B4810B50168002479B10A4A15
:102200000A4B02EB8102491E52F8044D1360016033
:102210002046FEF709FC10B90548FFF7B3FD20463C
:1022200010BD00004C0100206C0C0020ADDEADDEC6
:102230007800030000487047408100402DE9F74FC7
:10224000904607004FF0000502D13448FFF79AFD91
:10225000334C4FF4803BC4F808B3324EB07818B119
:102260002E48801DFFF78EFD706818B12B4809308D
:10227000FFF788FDDFF8B0A077605FEA08004FF055
:1022800000094FF00108AAF1040724D001282FD03B
:10229000022829D021481D30FFF774FD86F80280FE
:1022A000C4F840910199294489B239603F68C4F863
:1022B0004480DAF80060D4F8400118B117482B3098
:1022C000FFF760FDAF4215D3AE4201D3BE4221D32A
:1022D000124833301CE0C4F84480DAF80050C4F8E7
:1022E0004080C4F84091D9E70F48001D0568D5E744
:1022F0003D68D3E7BE4201D2012000E00020B54294
:1023000001D8012100E00021884203D103483E307A
:10231000FFF738FDC4F804B3BDE8FE8F8600040063
:1023200000800040240100204485004000487047A0
:102330004880004070B5144C01266660E660666413
:1023400012480025056011483C30006810B1104863
:10235000FFF718FD4FF0FF30C4F80803C4F84051F0
:102360000A490420083108600A4845600670457033
:1023700085700820FEF772F94FF0E0214FF480706D
:10238000C1F8000170BD00000080004008850040D9
:102390004700040024010020014800787047000035
:1023A000240100200349012008600349002008702F
:1023B00070470000008000402401002070B50748ED
:1023C00001250561C560064C002608206660667020
:1023D000FEF744F9A670257070BD00000080004033
:1023E00024010020014840787047000024010020AB
:1023F0000FB408B50399002904D004AA00926A46D4
:1024000000F00FF801B05DF814FB10B582680446C7
:10241000002A05D0D4E90403216898470020A06071
:1024200010BD2DE9FC4791460C00804676D014F88B
:10243000011B39B125290ED04046FEF78FFF2078C9
:102440000028F4D198F80C00002867D04046BDE879
:10245000FC47FFF7DABF0020012221782B291BD08F
:102460002D2902D0302908D102E040F0010001E01E
:1024700040F00200641C002AEFD100252A290ED06A
:102480002178A1F130020A2A11D205EB850201EB75
:102490004205641C303DF1E740F00400EAE7D9F85A
:1024A00000100B1DC9F800300968641C0D44217828
:1024B00000232E290BD114F8011FA1F130020A2AA2
:1024C00005D203EB830201EB4203303BF3E76C29B7
:1024D0000DD068290BD0692921D00BDC252918D013
:1024E000582931D063290ED0642915D117E014F88A
:1024F000011FECE7702969D0732932D075291BD0F0
:10250000782909D120E0D9F80000011DC9F8001090
:1025100001784046FEF722FF641C90E76CE0D9F892
:1025200000100A1DC9F800200968CDE900500A22F0
:102530004046FFF797F8EFE7D9F800100A1DC9F8F1
:10254000002009680A2206E0D9F800100A1DC9F81F
:10255000002009681022CDE90050404603F066FED5
:10256000DAE7D9F8001000270A1DC9F800200E6824
:10257000C00705D112E04046761C7F1CFEF7EEFE38
:1025800031780029F7D104E0202140466D1EFEF786
:10259000E5FEBD42C0D9002DF6D1BDE74EB13046B3
:1025A000FDF724FF074604E0202140466D1EFEF79C
:1025B000D5FEBD4206D9002DF6D103E04046761C7B
:1025C000FEF7CCFE31780029F8D1A5E7D9F8000054
:1025D000011DC9F80010056830214046FEF7BEFE17
:1025E00078214046FEF7BAFE08200021CDE900011F
:1025F000034610222946B0E7BDE8FC872DE9FF41DC
:102600001C46DDE90A7815460E46684600F0AAF831
:1026100046EA450141EA840141EA072242EA0841CB
:10262000009A00EB8200C0F80017BDE8FF812DE999
:10263000FF411C46DDE90A7815460E46684600F063
:102640009FF846EA450141EA840141EA072242EA4D
:102650000841009A00EB8200C0F80017BDE8FF8136
:102660002DE9FF411C46DDE90A7815460E4668460D
:1026700000F094F846EA450141EA840141EA072264
:1026800042EA0841009A00EB8200C0F80017BDE85A
:10269000FF812DE9FF411C46DDE90A7815460E460B
:1026A000684600F089F846EA450141EA840141EABA
:1026B000072242EA0841009A00EB8200C0F80017A6
:1026C000BDE8FF811CB5002100910B46012201915C
:1026D000FFF7C6FF1CBD1CB5002100910B4601226F
:1026E0000191FFF7D6FF1CBD1CB500220B460092DE
:1026F00011460192FFF7B4FF1CBD1CB500220B462A
:10270000009211460192FFF7C4FF1CBD1CB50021C9
:1027100000910B46012201911146FFF7A1FF1CBD5C
:102720001CB5002100910B46012201911146FFF7D3
:10273000B0FF1CBD13B50C46684600F021F80099A7
:1027400000EB8101D1F8002722F44032C1F80027C4
:10275000009900EB8100D0F8001741EA0441C0F86D
:1027600000171CBD0168202902D24FF0A04070471D
:1027700001F01F0101600148704700000003005094
:102780000168202902D24FF0A040704701F01F01DC
:1027900001600148704700000003005001682029D3
:1027A00002D24FF0A040704701F01F0101600148C4
:1027B00070470000000300500168202902D24FF04A
:1027C000A040704701F01F01016001487047000000
:1027D0000003005001B56846FFF7D2FFD0F810059E
:1027E0000099C84000F0010008BD01B56846FFF738
:1027F000D5FF009A01219140C0F8081508BD01B528
:102800006846FFF7D9FF009A01219140C0F80815EA
:1028100008BD38B501240090684631B1FFF7A2FF2A
:1028200000998C40C0F8084538BDFFF79BFF009920
:102830008C40C0F80C4538BD1CB5094C0144D4E9A6
:102840000034CDE900346C4606E000BF54F8203077
:10285000D3F81035401C08C28142F7D81CBD0000D7
:1028600044630000034908B5084400210160006882
:10287000009008BD0060004002494058012800D087
:1028800000207047006000402DE9F041204D1646C1
:1028900088460746082801D3042035E0B8F1000F28
:1028A00003D0202E03D906202EE003202CE038464A
:1028B00001F0D2F9032801D3092025E0384600F0C1
:1028C0008FFF032801D30A201EE000F0BFFC02287E
:1028D00001D2082018E000F043FE0446067040785C
:1028E000324640F0010060704146A01CFDF75AFDE1
:1028F000F8B2214601F0B2F910B10120BDE8F08133
:102900000448FFF73FFA0F2028700020F6E7000088
:10291000E0000020FC00050070B50E4C06460125C5
:1029200020880DA105EB004002F0EEF8FEF785FED1
:102930001049012208703046FFF7A6FF002807D192
:1029400020880DA105EB0040BDE8704002F0DCB826
:1029500070BD00006401002047617A656C6C2074D2
:1029600072616E736D697373696F6E206661696CF5
:1029700065640000000000205458206669666F20DE
:102980006572726F722000002DE9F84380462020A6
:102990001B4F11F0FF0F4FF0010500901DD06A464C
:1029A0001849404600F06AF828B9388816A105EBA6
:1029B000004002F0A9F8009878B112480024067887
:1029C00005FA04F03042204602D0FEF7ADFA01E0ED
:1029D000FEF7A2FA641C042CF2D3FEF72EFE0E4979
:1029E000012208704046FFF74FFF002805D13888C4
:1029F0000AA105EB004002F087F8BDE8F88300006B
:102A000064010020680100205258206669666F202A
:102A10006572726F7220000000000020545820661A
:102A200069666F206572726F7220000010B500F049
:102A3000D1FC18B1BDE8104000F004B8BDE810406A
:102A400000F0C6BB7047000010B50B4C606928B1A0
:102A500000F076FA0004000C02D005E0022008E045
:102A6000002000F087FD18B100F0C6FB012010BD6A
:102A700011202070002010BDE00000202DE9F04161
:102A800016460F46044600F0ABFE154D48B157B14F
:102A9000204600F0B1FE00783168814205D2062060
:102AA0001AE00B2018E0032016E0204600F09AFE02
:102AB00004000DD0A01C0BD02278A11C3846326037
:102AC000FDF770FC204600F041FD0120BDE8F081DB
:102AD0000448FFF757F90F2028700020F6E70000A0
:102AE000E000002026010500014800697047000051
:102AF000E00000200148007870470000E00000205E
:102B0000704700002DE9F0411D4D064600241D4888
:102B10002C70AC610460446084601B4800F0B8FB1A
:102B2000686140B3042000F029FA05F11C0029690E
:102B300000F048F80746304600F098F800EA07062B
:102B4000002000F079F80640012000F0A5F80640CA
:102B5000022000F059F80640002000F0BFF80640BF
:102B6000012000F02BFE0020EC6000F0E9FC16B123
:102B70000120BDE8F081012028700020F9E7000065
:102B8000E000002088090020F11B000070470000D1
:102B90000B48C268002A11D0012080F31088002160
:102BA00011600846C2F8041002EB8003401C9960D3
:102BB00099641028F8D3002080F310887047000033
:102BC000E000002010B50F4C6269527D0AB102206E
:102BD00014E010290FD871B178B10A46216101467D
:102BE00008481C30FDF7DEFB064821691C3000F068
:102BF000D9F9012010BD072000E00320207000203B
:102C000010BD0000E00000200A4910B54B690246E3
:102C100001205B7D0BB1022004E0012A05D0022ACD
:102C200004D00E200870002010BD002000F038FAFB
:102C3000012010BDE00000200A4910B54B69024692
:102C400000205B7D0BB1022003E032B1012A03D0EA
:102C50000E200870002010BD012000F09DF9012019
:102C600010BD0000E000002000F0BEBB10B540B178
:102C7000012808D002280BD0064905200870002042
:102C800010BD012000E0022000F0B4FB012010BDC7
:102C90000020F9E7E0000020014610B500200729D8
:102CA00014D2DFE801F0040F06080A0C0E0004201D
:102CB00008E0FC2006E0F82004E0F42002E0F02028
:102CC00000E0EC2000F0E4FF012010BD02490E20DE
:102CD0000870002010BD0000E00000200A4910B577
:102CE0004B69024600205B7D0BB1022003E032B14C
:102CF000012A03D00E200870002010BD012000F032
:102D0000D1FF012010BD0000E000002000B5054902
:102D100020B1C860FFF73CFF012000BD0320087010
:102D2000002000BDE000002010B501F0ADF903491E
:102D3000002008610249087010BD0000E009002071
:102D40000C0100202DE9FE434D4800684D4C012840
:102D500002D04D48006828B960680078202801D862
:102D6000012100E00021494E03204FF0000830709F
:102D70004348C4F8008008300568424F183F89B3C3
:102D8000006841490839086002A8CDE900043C48C0
:102D90000C30026801232946184602F0E9F810B306
:102DA000012805D0022821D0032855D0384851E009
:102DB000029818B136481C38FEF7E4FF284602F0A6
:102DC00037FA18B932481B38FEF7DCFF01F090F9EA
:102DD000B97D0023CDE900017068EAB290F91610C0
:102DE00018461CE01EE02A48113833E0029818B952
:102DF00027480D38FEF7C6FF284602F019FA18B921
:102E000023480C38FEF7BEFF01F072F9B97DEAB233
:102E1000CDE900017068012390F91610029800F0C6
:102E200077FB19E000F056FE30B101F061F9014680
:102E3000BA7DE8B200F03EFB0023CDF800801A46D0
:102E400019461846CDF8048002F092F8042803D001
:102E50000F480F30FEF796FF206838B101206075EB
:102E60000C48206104203070BDE8FE8301F00CF9AD
:102E700084F81580C4F8108000F00EF8F4E7000024
:102E800000140040E0090020341500400C0100202F
:102E900044060900312F000070B5FFF745FF1F4DB4
:102EA000012028701E4801681E4A21F0FF011269A6
:102EB0001143016002F0C6F91A4C4C3410B302F011
:102EC000C1F9032802D01848FEF75CFF022001F088
:102ED00019FB002001F06EFB02F0B4F9032803D0C7
:102EE00011480830FEF74EFF2878012803D00E481D
:102EF0000E30FEF747FF02202870002020610B48AB
:102F0000E06070BD01F0DCFF0228DFD302F0C2F800
:102F100060600028DAD10448401FD5E70C0100208A
:102F20003015004094090020F4050900452D0000EB
:102F3000024905200870FFF7AFBF00000C01002018
:102F40000148006A7047000094090020034910B549
:102F5000086200F09DFD0249086010BD9409002040
:102F60001C150040034910B5486200F091FD02496C
:102F7000086010BD940900202015004004494877DE
:102F800004490A6822F4E02242EA004008607047DF
:102F90009409002018150040014908767047000088
:102FA0009409002070B50C00054602D10748FEF7D1
:102FB000E9FE1DB90548401CFEF7E4FE0448C0E9DF
:102FC0000145BDE870400020FEF778BFB30309005B
:102FD000F809002010B500F07DFD044901F16402FC
:102FE00008B1C86800E08868106010BD940900202E
:102FF0001CB510494FF44070086002F023F9012815
:1030000012D0022810D0032813D1002000900346CC
:1030100002460146019001F0ABFF042809D0BDE84B
:103020001C400548FEF7AEBE0021084602F050F8ED
:10303000F3E71CBD08F5014048020900144981F876
:10304000310014490A6822F0FF020A6048B1114AAF
:103050000B1D0832012807D002280ED00E48FEF7BB
:1030600091BE086808607047086840F00100086079
:10307000FF20106040F2071007E0086840F00200EF
:1030800008604FF6FF701060044818607047000039
:1030900094090020341500402E040900211001007D
:1030A000044981F83200044908B1012800D10860C0
:1030B0007047000094090020101500402DE9FF41E1
:1030C0003E480068012802D03D48006830B93D48BC
:1030D00040680078202801D8012700E0002700F090
:1030E000E5FB384C0126183C00B9266102F0AAF82D
:1030F000012802D03448FEF745FE344D6868007D53
:1031000018B13148401CFEF73DFE00F0BDFFEFB3A3
:103110000121084601F0DCFF20B1012828D0022857
:1031200026D10FE000F0E4FF064601F0E9FEC7B249
:1031300001F0E0FE8446A07D0021CDE90260CDE9EA
:1031400000710DE000F0D4FF804601F0D9FEC7B257
:1031500001F0D0FEA17DCDE90076CDE90281844663
:1031600068686289218990F91630604600F0B2F9EA
:10317000FEF79EFEE06013484C3840696060FFF740
:1031800029FF04B00020BDE8F04100E001E0FEF7B7
:10319000ADBE6E7000F09EFC00280CD000F0A8FFC1
:1031A000054601F0ADFEA27D04B02946BDE8F04120
:1031B000C0B200F07FB9BDE8FF81000000140040FC
:1031C00034150040E0090020370709000C010020F9
:1031D00010B5012080F310880648417D29B181781F
:1031E00019B90121817000F02FFB002080F31088B5
:1031F00010BD0000C809002070B5124C607D002889
:103200001ED100F0BDFA04F13005A86810B90E48CF
:10321000FEF7B8FD686818B90B48401CFEF7B2FD10
:1032200002F036F818B10848801DFEF7ABFD00200B
:1032300002F04EF801206075BDE8704000F004BB5C
:1032400070BD0000C8090020CE02090001F064BE74
:1032500030B50D4D85B0687D002813D000F032FBED
:1032600000F012FF0024AC706C7505208DF8000092
:10327000684601F0D1FD0548047005B0BDE8304056
:10328000FFF7B6BE05B030BDC80900200C01002014
:103290002DE9F0410546012080F31088484E4FF09B
:1032A00003080024707086F80080B4707460348164
:1032B0007481F46007463461347506F11800747542
:1032C000046044608460C4600461047518308460E4
:1032D0004460FFF72FF8284601F0D8FD01F01EFEEC
:1032E000002001F0E7FF06F13000FEF711FE00219B
:1032F0000820FDF705FA00210120FDF701FA012160
:103300001520FDF7FDF9012000F074F8A6F1340551
:10331000FF202861042068772A4929622A496962C6
:1033200085F82870022185F8291085F82A8085F80B
:103330002B00052085F82C00062085F82D0007209D
:1033400085F82E00082085F82F0085F8304085F894
:10335000311085F83270692045F8140B1E20286062
:103360004FF4167045F8100C022000F069FC0F2095
:1033700000F06CFCEC802F716F712C72204601F014
:10338000C5FD7078012802D01048FEF7FBFC3770AD
:10339000B470746034817481F46034610C483475A5
:1033A00074758460447000F0EBF90820FDF74BF968
:1033B0001520FDF748F984F310880148BDE8F08135
:1033C000C809002004070A0D05080B0E9F0209001A
:1033D0000C0100200348407D08B100207047012007
:1033E00070470000C8090020014948837047000069
:1033F0009409002010B5012181F3108807490A784B
:10340000824204D04870487D28B100F01DFA0020A7
:1034100080F3108810BD00F003F8F8E7C809002019
:1034200030B5224D85B02878697888423BD008B9FC
:1034300000F0A6F9687808B9FFF7DAFD1C48002407
:10344000046000F021FE19481830046044600461F3
:103450008460C4602878012802D0022808D015E0D2
:1034600001F0F0FE90B10021084601F031FE0DE0C0
:10347000FFF75AFC01F0E6FE032807D10023009471
:103480001A4619461846019401F072FDFFF7A2FD95
:103490006878287004208DF80000684601F0BCFCB4
:1034A000012005B030BD0020FBE70000C809002066
:1034B00054F5014000B585B006238DF806208DF83F
:1034C00005108DF804008DF80030684601F0A4FC6A
:1034D00005B000BDF0B585B00DF1280C9CE8F000FA
:1034E0008DF80C308DF80D404FF0000C0190ADF8C8
:1034F00008108DF80E508DF800C0ADF80A208DF838
:103500000F608DF81070684601F086FC05B0F0BDC4
:1035100070B586B00226DDE90A458DF808108DF8F1
:10352000092001908DF80A308DF800608DF80C505C
:103530008DF80B40684601F06FFC06B070BD0000CE
:1035400001498860704700000C01002010B501217E
:1035500081F3108801F008FD002080F3108810BD71
:1035600010B5012080F3108801F000FD002181F3E7
:10357000108810BD10B50446082802D30348FEF792
:1035800001FC0348204490F8280010BDAD03090059
:103590009409002070B5082819D20F4A024482F815
:1035A00028108207D40EFF22A240D243042801D261
:1035B0000A4D01E0094D2D1D28681040286008467D
:1035C00000F054FA2968A0400843286070BDBDE8A7
:1035D00070400348FEF7D6BB940900202415004034
:1035E000A703090010B51B4C00206070FEF74CFCCF
:1035F00019490860FEF75CFC1849887501F022FE45
:10360000012807D001F01EFE022802D01448FEF760
:10361000B9FB002000F076FFFEF70CFE11490860B0
:103620006068091D40680860A068002811D0007813
:1036300020B1FEF7FFFDA16800F0C2FBA068017990
:10364000002906D000F090FBA068BDE8104000F013
:1036500099BB10BD0C01002008150040C8090020CE
:103660009706090050F5014010B501F097FD0028BC
:1036700020D0114800210181418101F041FC0F4916
:10368000086001F03DFC012181400C48001D0268EA
:1036900022F0FF021143016001F02CFC064C1834AB
:1036A000206001F021FC60600548E060BDE810404A
:1036B000FFF798BF10BD0000C80900202C1500407E
:1036C000BD3000001548002101600121016014484F
:1036D000016821F480710160016821F00F01891DEA
:1036E0000160016821F4702141F440310160001D46
:1036F000016821F000710160016841F08071016092
:10370000016821F0FF0141F020010160016821F40E
:103710007F4101600120FCF796BF0000FC1F0040C4
:103720001415004070B5134C1348A16800F056FE04
:103730006060114C4C3C607FFFF720FC206AFFF773
:1037400005FC606AFFF70EFC0025601990F8281050
:103750002846FFF71FFF6D1C082DF6D3074914F804
:10376000300F08606078FFF769FCA078BDE8704012
:10377000FFF796BC0C010020E00900200C1500406A
:103780000C4910B5002008600A484FF440744C38CA
:103790000460FFF797FFFEF7C9FD0649083108608E
:1037A000091F05480860034850380460BDE8104010
:1037B000FFF7B8BF54F501400411004010B50446AE
:1037C0000448406810B90448FEF7DCFA0348047561
:1037D00010BD00000C0100206E040900E00900206B
:1037E00001F026BD10B5012181F3108801F023FD01
:1037F000002181F3108810BD01F020BD0349012292
:10380000086101460248FEF719BD0000C809002002
:103810009D52000070B50C4601F05AFD074D286915
:10382000A04202D30648FEF7ADFA28690122211A08
:103830000448FEF703FD0020286170BDC809002080
:10384000D60609009D52000010B5FEF7A5FD01281F
:1038500022D101F037FD10B11048FEF793FA002293
:1038600064210F48FEF7EAFC0E48007F80B90E483D
:103870000121016000220007C0F80021016000BFA3
:1038800000BF00BFAFF30080D0F800110029FBD0CB
:10389000BDE81040FEF786BD10BD0000B40609006B
:1038A0009D5200009409002014050040044810B502
:1038B000006918B9FEF796FD002800D0012010BD60
:1038C000C809002010B5FEF767FD01280ED0FEF7ED
:1038D00075FD0748007F10B901208107486000206E
:1038E00001F0F6FC024900203431486010BD0000B0
:1038F000940900200B4810B54068407D30B101208C
:1039000000F058FE08490889401C0881074900203A
:1039100008600548343803C8BDE81040091A002083
:10392000FFF778BF0C010020C809002054F50140C2
:1039300070B586B0FFF7BAFF494D4A4E05F1340421
:1039400058B100F0BDF8A078002869D0FEF7F2FA6F
:1039500006B0BDE87040FFF77BBC2078012802D09C
:10396000022804D008E000F0E1FE28B170E03078D1
:1039700004286DD003286BD0FEF7DCFA00F0A0F825
:10398000A07868B1FFF764FC01F09AFA022840D3EE
:1039900003208DF80000684601F03EFA06B070BDC5
:1039A000FFF73EFD20B100206968FFF733FFEBE72A
:1039B0002078F0B1012816D0022817D02A48FEF747
:1039C000E1F9687E0128DFD100F084F80028DBD11E
:1039D0002078D8B1012811D00228D5D022481A3039
:1039E000FEF7D0F9D0E700F081F8EAE700F002F93D
:1039F000E7E700206968FFF70DFFE2E701F022FC2E
:103A00000028C1D101F09EFB0028BDD1FFF75AFF6D
:103A1000BAE706B01448BDE870403630FEF7B2B9D8
:103A20002078022808D0FEF785FA696806B00020E1
:103A3000BDE87040FFF7EEBE3078042808D00328B8
:103A400006D0FEF777FA06B0BDE8704000F0D2B8B5
:103A5000686806B04008BDE87040FFF7CFBE0000C0
:103A6000940900200C010020D0040900024610B582
:103A70000020014622FA01F303F00103C1F107041B
:103A8000A3400343491CC9B2D8B20829F2D310BDE0
:103A90002DE9F0410024064625461827E80026FABD
:103AA00000F0C0B2FFF7E2FF694207EBC1018840B6
:103AB00020436D1CEDB20446042DEFD3BDE8F08128
:103AC0000348416809B1491E4160FFF783BA00000D
:103AD000C809002004480178022902D04068002863
:103AE00000D0012070470000C80900202DE9F041F6
:103AF00086B000F0C9FA01F0A5FB3A4D05F1340497
:103B000020B3688BB0B3218981423BD301210020CF
:103B100001F0DEFA01F0EEF926898046648901F0B1
:103B2000EFF9074600F0E4FA014601208DF80000A5
:103B3000ADF808608DF80C70CDF80480ADF80A403F
:103B40008DF80D10684601F067F944E001F0B8F90E
:103B5000022840D3FFF7BEFF68B1FEF7C1F9D0BB22
:103B6000287E20B9FEF7A4F9E168884233D1FFF737
:103B70007BFD30E006E0E068FEF7A0F90020FEF7EC
:103B8000B5F9F4E7FEF72EFC10B11748FEF7FAF886
:103B9000FEF77AF915490968884202D06089401C0D
:103BA000608113484078A0B9FFF794FF88B101F015
:103BB000A7F9064600F09CFAA17D8DF806108DF855
:103BC000050007228DF800208DF80460684601F09A
:103BD00023F9FFF707FD296806B00120BDE8F04191
:103BE000FFF718BE940900207C0509000815004065
:103BF0000C01002070B50024FEF746F90D4D296830
:103C0000884207D0FEF740F92860FEF751F90A49CB
:103C1000012488750948641E0078044201D1FFF729
:103C20003BF9054834384168BDE870400020FFF793
:103C3000F1BD000008150040C80900200C0100205B
:103C40000149C860FFF7C6B994090020014988609E
:103C5000FFF7C0B99409002001F0FABA10B50122AB
:103C600082F3108801F001FB58B10848817819B936
:103C7000407D08B1FFF7E8FD002080F310880120A7
:103C800010BD002080F3108810BD0000C80900207E
:103C9000024981F830000249086070479409002009
:103CA0000C15004001490877704700009409002076
:103CB00070B51149114A0025487802EB0010027BCB
:103CC00022B10F4AD2F80C2102B10125807A087086
:103CD000012000F0DFFB0B4C1DB1A068806800B133
:103CE00080476068002806D00179002903D0BDE82C
:103CF000704000F01BB870BD040A0020A4630000EF
:103D0000001000402C01002007480069012805D060
:103D1000022805D0032805D100F09AB800F04CB96C
:103D200000F0E4B870470000040A0020827B002104
:103D300093000B4A1344C3F81019C37B02EB8302B0
:103D4000C2F81019427B0121837BC07B01FA02F289
:103D500001FA03F3814003481A430A4302607047A3
:103D600000F0014008F501404279054BC07901217E
:103D700003EB80000AB101667047016370470000E1
:103D80000060004082680021C2F84011C17B094AEE
:103D9000CB0009490B44C3F81025C37B826801EBB3
:103DA000C301C1F81425C17B012088400349086084
:103DB000704700001011004000F0014004F5014080
:103DC0002DE9F0410746886800260C46C0F840619E
:103DD0008868097B1A4D00F5A07005EBC101C1F898
:103DE00010056278E178207B00F08EFC607B05EBAB
:103DF000C000C0F81075617BA06805EBC101C1F877
:103E000014051048C0F80C61C0F81061A17B0E4881
:103E100005EBC101C1F810056278E178A07B00F0E4
:103E200061FC217B0120627B00FA01F100FA02F2C1
:103E30001143A27B9040014304480160BDE8F0813A
:103E400000F00140001000400C11004004F501405A
:103E50002DE9F0411F4E02200025307003207070C4
:103E600075603575B0691C4C401CB061C4F80C51CC
:103E7000C4F80051C4F81051C4F80451C4F82851D2
:103E8000C4F80052681EC4F808030120FCF7F1FBD7
:103E9000124FB868007D50B1114800684042B075BB
:103EA000C4F81C510120A0610E49800208600C4832
:103EB00044380068F168884202D00B48FDF762FF81
:103EC000B868C068002802D0BDE8F0410047BDE8EE
:103ED000F0810000040A0020001000402C010020A6
:103EE0004815004008F5014051040A0010B52D4C5A
:103EF000D4F80C01012802D02B48FDF743FFD4F879
:103F00001001012803D02848401CFDF73BFFD4F8DE
:103F10000001012803D02448801CFDF733FFD4F8AA
:103F2000040118B12048C01CFDF72CFF0020C4F884
:103F30000C01C4F81001C4F80001C4F80401C4F86D
:103F400008010221C4F800120121C4F80813082254
:103F5000C4F80423154A0323154C137010755060E0
:103F6000606890B1027912B1FFF7E0FE0DE00278CF
:103F70005AB1027B437B807B01FA02F201FA03F320
:103F800081400C481A430A430260A068006900B1EE
:103F90008047A0688068002802D0BDE81040004734
:103FA00010BD000000100040F3030A00040A0020C6
:103FB0002C01002008F501402DE9F0412A4DD5F8EB
:103FC0000001012802D02948FDF7DCFED5F80401E4
:103FD000012803D02548401CFDF7D4FE2448016881
:103FE000244801700021C5F80011C5F80411C5F876
:103FF0000811491EC5F808130126C5F80463816835
:104000001D4F097D09B1B1023960446814B32079AC
:1040100000B3617BDFF86480A06808EBC10100F5A4
:10402000A070C1F810056279E179607B00F06CFB4B
:10403000607B06FA00F03860207B114908EBC00075
:10404000C0F810156279E179207B00F04BFB207BF2
:1040500086403E600B480649091FC06808600B2077
:10406000C5F80002BDE8F08100100040BD030A0061
:10407000081500402C01002004F5014000F001402B
:104080000C110040040A002070B50120FCF7FCFA76
:104090000120FCF7EEFA144C4FF0FF30C4F808038F
:1040A0000026C4F80062C4F8106101202061A061FC
:1040B0000E4D2878012813D0022813D0032811D0E0
:1040C0005FF00100FDF74CFFC4F810612E706E75B3
:1040D000002000F0DFF9BDE870400120FCF7EABAEB
:1040E0000620EFE70220EDE700100040040A002060
:1040F00001480078704700002C01002001F03F01CA
:104100004FF4003343EA0121830009481844C0F802
:104110001015D0F810150AB941F48011C0F8101527
:10412000D0F8101541F00301C0F8101570470000D9
:104130000060004008480069012806D0022806D027
:10414000032806D00548FDF71DBE00F095B800F025
:1041500007B800F0F1B80000040A002033050A0097
:104160002DE9F047DFF8F0800421012088F80010E5
:10417000D8F81810491CC8F81810FCF77AFA374814
:104180000068374D2870374C0026C4F80C61C4F81D
:104190000061C4F81061C4F80461A868DFF8C89031
:1041A0000127007DA0B1304808380068400502D4DE
:1041B0002E48FDF7E7FD294840300068404288F866
:1041C0001600C4F81C61A7614FF48061C9F80010A3
:1041D000D4F8000118B125480930FDF7D3FDD4F813
:1041E0000C0118B121480A30FDF7CCFD4FF0E0205A
:1041F000B046D0F8000210F0020F03D01B480B307D
:10420000FDF7C0FD6E68CEB13078B8B1C4F80C814E
:10421000717B184A164802EBC101C1F8100572788B
:10422000F178707B00F05EFA707B0F4907FA00F0BE
:10423000091F0860F07B8740C9F80070A868C06853
:1042400000B18047A868417D002903D00349006878
:10425000091F0860BDE8F087040A00200815004027
:104260002C0100200010004008F50140C0040A00A5
:104270000C11004000F001402DE9F041294C0026CE
:10428000C4F80C61C4F80061C4F81061C4F8086196
:10429000C4F80461012004F58074FCF7EAF90820F1
:1042A000C4F804020125C4F808520720C4F800012C
:1042B0001D484468002C32D0207920B1207B1B4956
:1042C00005FA00F008602078002828D0A068C0F81F
:1042D0004061A17B164FA06807EBC10100F5A070FB
:1042E000C1F810056278E178A07B00F00DFAA068B3
:1042F000C0F84061E17B0F4807EBC101C1F8100530
:10430000E17BA06807EBC101C1F81405A17B05FAA8
:1043100001F0E17B8D4005492843091F0860BDE895
:10432000F0810000001000402C01002008F5014041
:1043300000F001400C11004070B5234CD4F80C0182
:10434000012802D02148FDF71DFDD4F810010128F5
:1043500003D01E48401CFDF715FDD4F800010128CC
:1043600003D01A48801CFDF70DFD0020C4F80C0195
:10437000C4F81001C4F80001C4F80401411EC4F8D7
:104380000813C4F80002124C626872B1117861B16E
:10439000557B012303FA05F1957BD27B03FA05F5E2
:1043A00093400C4A2943194311600B4903220870BA
:1043B0004A7048600875A0680069002802D0BDE80E
:1043C0007040004770BD000000100040F5040A0076
:1043D0002C01002008F50140040A002070B50646B3
:1043E0000C460120FCF750F9FFF74EFE244D2548FE
:1043F0002649C5E90146002404700326467044603E
:1044000004610475447584751F4808601E48F030C7
:10441000091F08601E48016821F0010141F0807108
:1044200001600120FCF746F9686838B3017909B9E1
:10443000017819B38168C1F808650422C1F8102514
:10444000027CC2F18102C1F8402540F20112C1F89C
:104450000022C1F804450122CA60C1F84041017937
:1044600021B142798179C079FFF748FE6868017807
:1044700021B142788178C078FFF740FE014870BDD5
:104480002C010020040A00201410004064F50140B3
:10449000741700402DE9F041174C00250746C4F879
:1044A0000052164E307803281CD0681EC4F808034A
:1044B000C4F80C51032070700120FCF7DAF800BF3B
:1044C000C4F80051C4F81051C4F804517560357532
:1044D000002F0FD00A488068006900280AD0BDE884
:1044E000F04100476FF00800C4F808030820C4F842
:1044F0000403E5E7BDE8F08100100040040A002055
:104500002C0100202DE9F0470746DFF89080224873
:104510004FF0FF3100EB0716C8F808130120FCF735
:10452000A8F81F4C0025DFF87C9065756770D9F8F6
:104530000800032F0268A2604168C4E90315A56161
:104540003068606019D2337AC8F80032C8F80C516C
:10455000C8F81051F37A14481BB10160006828B103
:1045600008E00260006828B9104801E00F48401DCB
:10457000FDF708FC717AC8F80413D9F80800007D2B
:1045800028B1022F03D10A49A575780208600120DD
:104590006075BDE8F0870000A463000000100040D3
:1045A000040A00202C010020041500409C020A008F
:1045B00004F501402DE9F05F404C824640486678A2
:1045C00000EB0617607D012802D03E48FDF7DAFBBC
:1045D000207D18B13B48401CFDF7D4FB012500218C
:1045E0002575DFF8E490A0466175032E47D2BAF135
:1045F000000F3CD1D9F80440BCB32279AAB38A4653
:104600000846A168C1F84001217BDFF8C0B0A0686E
:104610000BEBC10100F5A070C1F810056279E179DA
:10462000207B00F071F82A49C1F80CA1607B294970
:104630000BEBC000C0F810156279E179607B00F0E7
:1046400051F8217B627B05FA01F005FA02F108437B
:1046500021490860D9F80400204A81791268CA40CB
:1046600012F0010F01D18068056038680560022EE4
:1046700001D0012E07D1B97A88F8001003E0114863
:104680002530FDF77FFBD9F80800007D002813D006
:10469000022E11D110480068400503D409482A3081
:1046A000FDF770FB0E480068002805D1BDE8F05FFB
:1046B00004482B30FDF766BBBDE8F09F040A0020DC
:1046C000A4630000B8020A002C01002000F00140A1
:1046D000001000400C11004004F50140100500508E
:1046E00004150040064B03EBC0000AB1054A01E087
:1046F000044A303A02EB8101C0F8141570470000FB
:1047000000F0014060600040064B03EBC0000AB1BE
:10471000054A01E0044A303202EB8101C0F8141569
:104720007047000000F00140306000400348D0F8BE
:104730000401012800D00020704700000010004054
:1047400030B5124B01460020D3F81044224609E050
:10475000157A854205D1401C0A28F7DB4FF0FF305F
:1047600030BD5268002AF3D1421CF9D00872D3F848
:1047700010242AB152684A60D3F81024516030BD29
:104780000022C3F810144A6030BD00006405002008
:10479000F0B595B01C4615460F4608461A9E00F027
:1047A00019FB182109A8FBF716FE0E96CDE909544E
:1047B0000023082203A9384600F021FB0598069043
:1047C000BDF81000ADF81C00BDF81200ADF81E00D9
:1047D00000208DF821000398082600F0030001282E
:1047E00002D0022818D032E003983346850AC0F37D
:1047F000C2008DF8200003980FA9C0F38314A20013
:10480000384600F0FCFA09A8009006AB22460FA932
:10481000284600F03BFA1AE00398840DC0F3C2006A
:104820008DF82000082C01D2254600E008253346EB
:104830002A460FA9384600F0E2FA2E44641B09AB61
:1048400006AA29460FA800F073F9002CEAD13846D1
:1048500000F0C6FA15B0F0BD7047012001F056BB5C
:10486000084810B50178084A515C19B1001D01F0E3
:104870004FF802E00C3000F05DFFBDE81040002072
:1048800001F044BB6C0000201400002008B5034A6E
:1048900000924023024AFFF77BFF08BDF95B00004E
:1048A000640400200A4A012902EBC00007D0022953
:1048B00007D0032907D0042907D000207047022021
:1048C00070470420704700797047407970470000B6
:1048D0005C65000010B5FFF7C0FF04210348FFF737
:1048E0002FFF02490120487210BD00008000002007
:1048F0002DE9F0478CB0FCF741FD18B100200CB059
:10490000BDE8F087784C0020C4F81804BFF34F8F3F
:1049100060680290A5684FF00008284004EB800012
:1049200008E021680298814201D86160E6E72840EA
:1049300004EB80000C3002A9FCF728FF0028F0D11E
:1049400003AB029901EA050204EB8202491CD2681A
:1049500043F82020401C02910228F2D3039800F073
:104960000300022802D001284ED0A5E0039850226F
:10497000810D8946B2EB905F00D850210E4666F358
:104980009F5003900831594800F0DBF9070078D0B8
:1049900000F020FA4346082203A9384600F035FA11
:1049A000029908F1080A2940681A8000001D864211
:1049B00023D94D4D0C3530B1C2B204EB8101301A10
:1049C00090460C3104E02946F2B200259046284674
:1049D000C6B25346384600F018FA0AEB08032DB168
:1049E000324629464FEA070000F00FFA029909F112
:1049F000030001EB900002903AE004EB8101534682
:104A0000324638460C31EFE70398C0F3831106298C
:104A100000D3062161F389100390C0F38310801C3A
:104A20008100324800F08DF9070045D000F0D2F93E
:104A30004346082203A9384600F0E7F908F10808C0
:104A400000260FE00298434600EA0501401C04EBF3
:104A500081010290042238460C3100F0D6F908F1A9
:104A60000408761C0398C0F38310B042EAD847B11B
:104A7000D4F81054D4F8180468B1384600F0B0F9EE
:104A80002CE019E0687A012804D12A6828463946C2
:104A9000126890476D68002DF4D1384600F0A0F9F7
:104AA0000020FCF759F9D4F8180408B9029860609E
:104AB0000020FCF753F911E0D4F8104404E0216819
:104AC0002046896888476468002CF8D1084802218C
:104AD000008801EB004007A100F016F8FCF74EFC3F
:104AE00080F001000BE70000640500208C650000E9
:104AF000640100204261636B656E647320666C75AF
:104B0000736865640000000000231A4601F094B841
:104B100008B5012300926A4601F08EF808BD3EB543
:104B2000069C8DE81C0003236A4601F085F83EBD13
:104B30002DE9F0470E4680461C46924608293ED88D
:104B400094F80C90002020731946104600F0AEFF38
:104B50000025B54206D218F805201AA12046FDF717
:104B600047FC03E019A12046FDF742FC6D1C082D0F
:104B7000EFD317A12046FDF73BFC0025B54210D22C
:104B800018F80570FBF70AFC0068C05D10F03E0FD6
:104B900001D03A4600E02E220EA12046FDF728FC67
:104BA00003E00DA12046FDF723FC6D1C082DE5D385
:104BB00001222146504600F05BFF84F80C90BDE8CE
:104BC000F0870000202530327800000020202000EF
:104BD0007C0000002563000020000000104810B594
:104BE000FF218160002101604160C0F81814C0F805
:104BF000141480F820140B4800F0F0F800280DD1B0
:104C000009480A490A4B401AC108002003E000BFC6
:104C100023F82000401C8842FAD3002010BD000079
:104C2000640500208C6500008C6500005C65000058
:104C30005001002002480349401AC0087047000094
:104C40008C6500005C65000013B56846FCF7B8FF92
:104C500008B100201CBD0248009950F831001CBD6D
:104C60005C65000070B508480125D0F8104480F854
:104C7000205405E0657221682046496888476468C9
:104C8000002CF7D170BD0000640500202DE9FF471E
:104C900081460C9D00200C462F7B287398461646B3
:104CA0002946184600F002FF072E42D2DFE806F040
:104CB00004090F161F2A360049462846FDF798FBBF
:104CC00037E0494628462268FDF792FB31E0D4E9F7
:104CD000002349462846FDF78BFB2AE0A068009098
:104CE000D4E9002349462846FDF782FB21E0D4E9B8
:104CF0000201CDE90001D4E9002349462846FDF729
:104D000077FB16E004F1080007C88DE80700D4E936
:104D1000002349462846FDF76BFB0AE004F1080032
:104D20000FC88DE80F00D4E9002349462846FDF757
:104D30005FFB00222946404600F09AFE2F73BDE833
:104D4000FF872DE9F041858A80462D1F4819C01C38
:104D5000B0FBF5F0C6B24046FDF738F8041E19D096
:104D60000020207101206071E58000272546761E15
:104D7000C4F800800BE04046FDF728F860B1617987
:104D8000491C6171286005467F1CC0F80080B7424D
:104D9000F1D32046BDE8F081204600F002F8002063
:104DA000F8E72DE9F041457901466B1E002201E04C
:104DB0000968521C9A42FBD30F680146002605E0A1
:104DC00038460C68FDF721F82146761CAE42F7D331
:104DD000BDE8F0810121001DFCF7DCBFFDF72AB81A
:104DE00010B504460121001DFCF7EAFF10F0FF0F8B
:104DF00004D12046BDE81040FFF7D3BF10BD38B541
:104E000001240094FCF7A0FE38BD38B500240094BE
:104E1000FCF79AFE38BD000070B51A4C05462068B4
:104E200010B91948FCF7AEFFD4F8D4000A2803D310
:104E30001548401CFCF7A6FFD4F8CC0000EB80001E
:104E400004EB800115F8040B08712DCD8860CA6051
:104E50000B614D61D4F8D400401CC4F8D400D4F8E0
:104E6000CC00401CC4F8CC00D4F8CC1000200A2997
:104E700001D3C4F8CC004FF0E0214FF40010C1F88A
:104E8000000270BD200A00204A000B0010B504008B
:104E900002D10948FCF776FF084941F8CC4B0020C5
:104EA00041F874098867C8674FF0E0214FF400109B
:104EB000C1F8000110BD00003E000B00200A0020D8
:104EC00010B5074CD4F8D4000A2802D90548FCF7DD
:104ED00059FFD4F8D400C0F10A00C0B210BD0000E0
:104EE000200A002079000B000148C06870470000CC
:104EF000F80A00200148806870470000F80A002086
:104F00000148406870470000F80A0020014981F814
:104F100081007047F80A0020FDF794B870B5FDF7DE
:104F200097F800240E4E2546204600F049FD04F176
:104F3000080000F045FD3555641C082CF4D30948E1
:104F40000121057045608560C5600561456180F897
:104F5000805080F85850C56780F8811070BD0000FF
:104F600038010020F80A0020FDF79EB8FDF742B98D
:104F70002DE9FF4F81B0444FDDE90EA8032600253F
:104F8000F86F0C46AB4610B94048FCF7FBFE38788A
:104F9000032803D03D48401CFCF7F4FEF86FB946E7
:104FA0004178C8072FD199F8810060B30027019894
:104FB000E8B3039A584662F31700C1F3410161F365
:104FC0001F6009EB84018A6BCAF800B0C8F800B012
:104FD0000090904234D0204600F032FD051E07EAD2
:104FE00005072DD004F1080109EB810200999161B8
:104FF00004990D4223D0264E305D00B3204600F0C8
:1050000027F910B105E00127D1E720482830FCF747
:10501000B9FE204600F01EF9CAF80000BAF1000FF0
:105020000AD018B919482E30FCF7ACFE00E01BE09E
:1050300006F804B0022603E014483230F4E70126F3
:1050400077B1204600F022F9C8F8000018B11048E6
:105050000121015506E00C485830C8F8000001E075
:10506000C8F800B00DB107E004264C46D9F87C0022
:10507000FDF71AF8C4F87CB089F800B000F068F8C1
:1050800005B03046BDE8F08FF80A00202D010C0075
:105090003801002010B50C4C207810B10B48FCF7FB
:1050A00071FE00F0C1FC00280DD0FF220270417893
:1050B00041F00601417000214318491C9A702029D3
:1050C000FAD30321217010BDF80A002007010C005B
:1050D00070B51A4C05460E462078012804D00228E7
:1050E00002D01748FCF74EFEB5B12078012803D056
:1050F0001348401DFCF746FEE06818B91048801DB3
:10510000FCF740FEE068007820B1606800F098FC91
:10511000022502E0002500E004254EB1606800F0A1
:1051200099F8A168814203D005481D30FCF72AFE9A
:105130000020207000F00CF8284670BDF80A00200E
:10514000CC000C00014890F880007047F80A00205D
:105150002DE9F041104C207800281AD194F88000F5
:10516000002816D10825012600276069FCF7C6FF34
:1051700018B184F88060606920616069401C6061DA
:10518000082800D1676194F88000002801D16D1EC5
:10519000EBD1BDE8F0810000F80A002070B5224C88
:1051A000207810B12148FCF7EDFD94F8800000252F
:1051B000F8B12069606000F069F8A06018B91B4878
:1051C000C01DFCF7DFFDA0684078C00705D194F84A
:1051D000810010B10220E56009E0606800F028F865
:1051E000032806D200F020FCE06010B101202070FE
:1051F00002E02078002815D0A06818B90B482030AC
:10520000FCF7C0FD2069606004EB8000C17E491C92
:10521000C17684F88050C27EA068417862F3420172
:105220004170012070BD0000F80A002098000C00B9
:105230000830FCF763BF0830FCF770BF0830FCF79C
:10524000BDBF00000148007870470000F80A002048
:10525000FCF754BF70B50446FCF760FF050002D0B0
:10526000204600F0CDFB284670BD70B50E460446C2
:105270000025FCF7E7FE38B121463046FCF770FF09
:1052800010B1FFF765FF0125284670BDFCF796BFFA
:105290000148007870470000400100200448017870
:1052A000817041780170001D50F821000047000016
:1052B0004001002002498870487008707047000063
:1052C0004001002001484078704700004001002064
:1052D00010B50446022802D30248FCF753FD0248E9
:1052E000447010BD33000D004001002040580028DC
:1052F00000D00120704708B500224250405800906D
:1053000008BDD0F80403084000D001207047405881
:10531000002800D00120704708B5002242504058B4
:10532000009008BD002802D001498001084770475D
:10533000616300002DE9F0410E46804600F048FB15
:10534000204D0028404616D0FCF758F8284490F825
:1053500058008009032802D001280AD003E0404603
:10536000FDF738FA28B103214046BDE8F041FDF7CA
:10537000E1B90221F8E700F037FB002820D04046D1
:10538000FCF73CF80446104F4FF4807007EB8401A3
:1053900000EB8400D1F8102580B242F00102C1F880
:1053A0001025FDF75FFA002E0AD04046FCF726F8DC
:1053B00055F82000002803D00120A040C7F80403BE
:1053C000BDE8F0817C020020006000402DE9FC4136
:1053D000DFF8C080044608EB0400002790F9300095
:1053E0001346C0170E46401C01D008274FE0B07886
:1053F0001946C0F340022046FBF7DCFF0546401C7F
:1054000044D0B07841071CD4C0070DD06846009442
:10541000FDF7B6F9009900EB8100D0F8001721F0F4
:105420000201C0F8001707E00021737820460091C0
:105430000A460191FDF7FBF8164920466431FCF756
:1054400019FDB078800718D51348317800EB850036
:10545000D0F81025114B1A40C0F810254FF47C529B
:105460004FF4403302EA042203EA01410A43D0F830
:1054700010150A43C0F8102509E008EB0500327842
:1054800010F8581F41EA8211017000E004273846E5
:10549000BDE8FC817C02002000600040FFC0FCFFF2
:1054A00010B5FDF797F9002800D0012010BD0000CD
:1054B00070B5194D95F86A0008B1082070BD00203C
:1054C000411E2A18401CC0B282F830103028F8D390
:1054D00000242046FBF760FF641CE4B20C2CF8D3D8
:1054E0000D490024E0204C66A1F868400B4981F882
:1054F000000401264020891FC1F88002C1F8000184
:105500004FF4BE70FDF7AEF90549F007C1F804038A
:1055100085F86A60204670BD7C02002006E000E04D
:1055200000600040034890F86A00002800D0012085
:10553000704700007C0200200121B1EB507F01D1B7
:10554000012070470020704770B50D4600F0FAFA50
:1055500004000FD00020FBF7FFFB207920B10020D2
:10556000FBF7FCFB112070BD01202560207100209D
:10557000FBF7F4FB002070BD10B500F0E3FA002843
:1055800002D000210160017110BD000001490248F4
:1055900000F0E4BCE8020020002000402DE9F041CA
:1055A0000546007916460F4600EB40012D4A01EBF7
:1055B000C00102EB810494F82A1011B10820BDE863
:1055C000F081294951F820102868FFF7BDFF08B184
:1055D0001120F4E739462846FBF7D4FB66603869AA
:1055E000206030004FF001062FD03F7F4FF48E71C6
:1055F0002868FFF780FE4FF4A2712868FFF77BFE52
:1056000028681A49C0F8041328684FEA4711000BAC
:1056100040B2002806DA00F00F0000F1E02080F828
:10562000141D03E000F1E02080F800142868000B4E
:1056300040B200F01F0206FA02F14009800000F1BA
:10564000E020C0F88012C0F8001128680421C0F8DA
:1056500000150020A061E06184F8290044F8140FCF
:10566000A675ACE7E80200204C6300008000020051
:105670002DE9F047054600790B4600EB400101EBB0
:10568000C000234901EB8004284600F043F810B124
:105690001120BDE8F0874FF00008C4F82080A36017
:1056A000626184F828804FF48E7647463146286838
:1056B000FFF721FE28684FF00109C0F80890214645
:1056C000286800F0E7FB606800BBD5F800A00EE09A
:1056D00094F8280008B10F2716E031465046FFF72E
:1056E00005FE0028F4D02146504600F0D3FB216A85
:1056F00060698142F1D331462868FFF7F7FD002841
:10570000F9D02868C0F80C90C4F814803846C0E777
:10571000E8020020007900EB400101EBC0000449E1
:1057200001EB80004069002800D001207047000094
:10573000E80200202DE9F047044600794FF0000907
:1057400000EB400101EBC000254901EB8007206818
:10575000C0F80095786880B120682249C0F8081325
:1057600020680121000B40B200F01F029140400967
:10577000800000F1E020C0F880112068D0F80C25EE
:10578000D0F81485D0F80865D0F810554FF0FF31E7
:10579000C0F81415C0F80C152068C0F80815C0F83A
:1057A0001015501C02D01046FCF78CFFB8F1FF3FDB
:1057B00002D04046FCF786FF681C02D02846FCF762
:1057C00081FF701C02D03046FCF77CFF2068FFF799
:1057D000D3FE87F82A90C7F80490BDE8F087000050
:1057E000E8020020840202000149024800F062BC85
:1057F00014030020002000402DE9F0410546164624
:1058000000790F46154A00EBC00102EB810494F8C1
:10581000201011B10820BDE8F081114951F8201085
:105820002868FFF791FE08B11120F4E739462846B1
:10583000FBF7E3FA6660386920601EB1397F2846BD
:10584000FBF764FF28680821C0F800150020A0615C
:10585000E0610121606184F82010DCE7140300207E
:10586000506300002DE9F04704460E4600792049B8
:1058700000EBC00001EB800517463046FFF75CFEE9
:1058800030B1204600F036F820B11120BDE8F08795
:105890001020FBE76F61AE604FF490760027314631
:1058A0002068FFF739FD4FF4AC7841462068FFF7D8
:1058B00033FD2068AA686969C0F84425C0F8481516
:1058C000206801218160686878B9B146494620683E
:1058D000FFF71DFD064641462068FFF718FD064309
:1058E000F4D000B10F27002068613846CEE70000F1
:1058F000140300200079054900EBC00001EB800093
:105900004069002800D001207047000014030020E7
:105910002DE9F04704460079274900EBC00001EB70
:10592000800720684FF00009C0F80095786880B1C2
:1059300020682249C0F8081320680121000B40B2FA
:1059400000F01F0291404009800000F1E020C0F803
:1059500080112068D0F80C25D0F81485D0F808659F
:10596000D0F810554FF0FF31C0F80C15C0F81415E1
:105970002068C0F80815C0F81015501C02D0104659
:10598000FCF7A9FEB8F1FF3F02D04046FCF7A3FEAA
:10599000681C02D02846FCF79EFE701C02D03046E0
:1059A000FCF799FE2068FFF7E7FD87F82090C7F81D
:1059B0000490BDE8F08700001403002010030200EB
:1059C000024A002102EB800081617047F80A002042
:1059D0000449084490F93000082801DB0120704791
:1059E000002070477C0200200449084490F93000F0
:1059F000082801D201207047002070477C02002057
:105A000010B50446064890F8801021B10069A04204
:105A100001D1FFF79DFB03490020085510BD000090
:105A2000F80A00203801002010B5044CE06F00286F
:105A300002D1FCF7DFFBE06710BD0000F80A002090
:105A400070B5094D0446E86F10B90848FCF79AF99B
:105A500004F10801E86FFCF783FB002802D0002066
:105A6000E867012070BD0000F80A00202E020C003B
:105A700010B50C46017A052908D0407A38B108489B
:105A800008A102682046FCF7B3FC00E01AB106A1A9
:105A90002046FCF7ADFC2046BDE81040FCF7B5BC45
:105AA000B8000020257300000D0A000038B5C38837
:105AB0000D46044633B114A0009015A216A1284645
:105AC000FCF796FC217A05291CD0607A48B1A088A1
:105AD000FEF7E8FE164951F8202016A12846FCF7EB
:105AE00087FCA0880021FFF7AFF803461049207A11
:105AF000143951F8202001B02846BDE830400EA1ED
:105B0000FCF776BC38BD00001B5B306D0000000068
:105B10001B5B313B33316D0025734C6F6773206421
:105B2000726F70706564202825642925730D0A0042
:105B3000B8000020257300003C25733E2025733AF1
:105B4000200000000349884201D10348704700202B
:105B500070470000002000402800002070B501269A
:105B600070044FF0E0210025C1F88001084C40107E
:105B7000C4F84803C4F8080366602F20FFF7D2FB7F
:105B8000A660044C2F20A560FFF7CCFBA57070BD6C
:105B9000001001405000002070B5054688690C4691
:105BA00000284FF4847128460AD0FFF7A4FBD5F8EB
:105BB0001805626AE1688854606A401C606270BDC2
:105BC000FFF799FBD5F8180570BD1FB501238DF8B7
:105BD0000030CDE90121D0E90012684690471FBD91
:105BE0001FB501238DF800308DF808100192D0E91F
:105BF0000012684690471FBD70B50D4C0020D2B210
:105C00002070201D0B4D0378EB5C1BB1001DFFF7CE
:105C100029FE02E00C30FFF72BFD08B1FBF704F87A
:105C20006078002802D021780029FAD070BD0000E9
:105C300068000020140000202DE9F84F204D924606
:105C4000894606469846012269461846AF68FBF722
:105C500041FB58B3009800210446801C09E000BFB6
:105C600000EA07035AF8212005EB8303401C491C76
:105C7000DA604145F4D34FEA164AFBF769FC4AEA79
:105C80000041601C384005EB80003C4005EB84027D
:105C9000C160D06866F3C50068F3891069F39F207E
:105CA00020F00300401C20F00400D06095F8200490
:105CB00002E000BFFEF71CFE0028FBD1BDE8F88F14
:105CC000640500202DE9F84F1D4C00256846D4E9F5
:105CD00001A6FBF747FC002738B30023009A616850
:105CE0001CE0D1F800C00846944503D9ACEB020291
:105CF0000A6015E0A2EB0C0263440760D0F80CC008
:105D0000C1698146BCF1000F08D006EB030828F0FA
:105D10007F48C0E9018CC9F81C5005460029E0D134
:105D200028466160FBF77AFD03E02846FBF776FD25
:105D300010B15046FBF76AFBE770BDE8F88F000032
:105D4000500000200D4B10B5596831B102680C6845
:105D5000A24204D8A21A0A60C161586010BD0B4665
:105D600003E00B46C969121B21B10C689442F8D3B9
:105D7000A41A0C600260C161D86110BD50000020FF
:105D80002DE9F041144E77683D462C4603E08442ED
:105D900004D02546E469002CF9D11BE0D4B1A5421A
:105DA0000BD1F869706040B90C490120886000216E
:105DB000B160F0702F20FFF7B5FA2168E069E86163
:105DC00010B10268114401607068874202D001205E
:105DD000BDE8F0810020FBE75000002000100140EA
:105DE000F8B5064600240D462046FAF7B5FF68468A
:105DF00000F076FA68B10570084946609DF8000029
:105E000048700020FAF7AAFF1420FAF75EFC20463B
:105E1000F8BD04240020FAF7A1FFF8E7580300209A
:105E20002DE9F041194D6C68002C2CD01848002742
:105E30000068A968B846401A20F07F462068B04242
:105E40000CD82146361A0744E469087C20B181F851
:105E50001080886949698847002CEFD129786878D3
:105E6000814206D1401CC0B26870022801D185F879
:105E70000180064869780C3040F82170BDE8F04197
:105E80001420FAF722BCBDE8F08100005000002089
:105E90000415014070B50C4605464FF48E71FFF7AE
:105EA0002AFA216AA068415C206A401C2062C5F879
:105EB0001C1570BD1FB500228DF80020029181686D
:105EC00001914261D0E90012684690471FBD000071
:105ED0001FB50A4601788DF8001041680191017ADA
:105EE0008DF80810C0680390044850F82210083854
:105EF00050F82220684690471FBD00002000002077
:105F000001490120087070476800002010B588B072
:105F1000044620220E496846FAF744FA062000900B
:105F2000C01F0190029003904FF0EB7006900CB1EF
:105F3000084A00E0002269460748FCF74FF808B11C
:105F4000FAF772FE0448001F447008B010BD00004C
:105F500084630000015F00006C0000202DE9FF4712
:105F60000C4605464FF40071FFF7CBF901274FF4BB
:105F70000178002618B34FF4927949462846FFF776
:105F8000B5F9E0B149462846FFF7B5F9C5F80883E9
:105F900094F8290000B96F6002208DF80000D5F850
:105FA0008004C5F880040390A0690290E068019025
:105FB000A661E661D4E900126846904728E0042112
:105FC0002846FFF79EF918B34FF484712846FFF76F
:105FD0008DF9E8B121462846FFF7DEFD616AA06928
:105FE000884215D1E06938B1E268616AA061206930
:105FF000E6616662E06008E094F8290000B96F602D
:10600000C5F80883A661E268616A2046FFF7DDFDF6
:106010004FF48E7841462846FFF768F978B1206A38
:106020006169884202D294F8280020B3414628468C
:10603000FFF761F9616911B12046FFF73BFF4FF4AB
:10604000A27841462846FFF751F9002818D041466A
:106050002846FFF750F994F8290000B12F60A06995
:1060600000280DD0A661E268616A04B02046BDE850
:10607000F047FFF7AABD21462846FFF70BFFDEE7F2
:10608000BDE8FF871FB50A4601788DF8001041680A
:106090000191017A8DF80810C0680390044850F807
:1060A0002210083850F82220684690471FBD000093
:1060B000200000202DE9FF410C464FF49277054661
:1060C0003946FFF724F90026C0B139462846FFF7C4
:1060D00023F902208DF80000D5F88004C5F880046B
:1060E0000390D5F83C058DF80800E0680190A661A2
:1060F000E661D4E900126846904723E04FF48877C0
:1061000039462846FFF703F9E0B139462846FFF73C
:1061100003F9D5F83C15A069884213D1E06960B154
:10612000E268D5F8000220F02000C5F80002E0691E
:10613000A0612069E661E06001E0A661E2682046B6
:10614000FFF74EFD4FF4A27739462846FFF7DFF8F8
:1061500060B139462846FFF7DFF8A06930B1A66183
:10616000D5F83C152046E268FFF73AFD4FF49077EA
:1061700039462846FFF7CBF8002813D03946284681
:10618000FFF7CAF8606900280CD0D5F84C058DF8E7
:1061900000608DF80800A06801906661D4E90012E3
:1061A00068469047BDE8FF8110B5FAF75BFD08B17E
:1061B000FAF73AFD00210320FAF766FF08B1FAF773
:1061C00033FD4FF400410020FEF708FD08B1FAF757
:1061D0002BFDFEF77FFB09480321008801EB0040FF
:1061E00007A1FEF791FC00BFFEF782FB0028FBD160
:1061F000BDE810400120FAF74FBE00006401002006
:1062000047617A656C6C2041434B207061796C6FFB
:106210006164206578616D706C652E2044657669D7
:106220006365206D6F64652E000000002DE9F05F4E
:106230008346DDE90A4A994690460D4608460127FD
:1062400003E000BFB0FBF8F07F1C4045FAD2B9452F
:1062500000D94F465FEACA7012D18CB15FEA8A70EA
:1062600002D5B9F1000F01D0202607E0302605E065
:1062700031465846641EFBF771F80CB1A742F7D3BC
:106280005FF00106B9F1010F02D9A9F1010903E09C
:10629000B5FBF6F0404502D306FB08F6F2E7DFF85F
:1062A0003C9000BFB5FBF6F000FB165519F8001046
:1062B0005846FBF753F8B6FBF8F6002EF2D15FEA2A
:1062C000CA7009D0002C07D0A74205D22021584619
:1062D000641EFBF743F8F5E7BDE8F09F6663000036
:1062E0000A494A788B78521CD2B2934200D10022DC
:1062F0000B78934201D1002070470270487800EB80
:10630000400001EBC000001D704700005803002052
:106310000D0E0F100B0C1819100200203002002077
:106320005C0200200B000300A90F00000C0003001A
:10633000A90F000018000300A90F000019000300B6
:10634000A90F000000000050000300508D55000010
:10635000E95700000300000038030020000000009F
:106360000338FDD870473031323334353637383959
:1063700041424344454600008D480000614800000A
:1063800059480000FFFFFFFFFFFFFFFFFFFFFFFF78
:10639000FFFFFFFF00000000000000000000D6012A
:1063A0000701000000100040101100400310000021
:1063B0000100000000100040000000000B0204007B
:1063C000000000000410004000000000070103016D
:1063D00000000000004040404040404040404141FB
:1063E00041414140404040404040404040404040AA
:1063F0004040404040050202020202020202020244
:106400000202020202202020202020202020200240
:1064100002020202020290909090909010101010D0
:10642000101010101010101010101010101010106C
:106430000202020202028888888888880808080800
:1064400008080808080808080808080808080808CC
:106450000202020240000000D56300004368616E42
:106460006E656C2025753A20253033752070616388
:106470006B657473207472616E736D697474656496
:106480002C2025303375207472616E736D697373BF
:10649000696F6E73206661696C65642E0000000090
:1064A0007761726E696E67006465627567000000EF
:1064B0001B5B313B33306D001B5B306D0000000017
:1064C0001B5B313B33316D001B5B313B33326D0065
:1064D0001B5B313B33336D001B5B313B33346D0051
:1064E0001B5B313B33356D001B5B313B33366D003D
:1064F0001B5B313B33376D00696E666F0000000037
:106500006572726F720000004750494F5445000099
:10651000505253005541525400000000554152540E
:106520004500000062616C6C6F632E6C6F675F6D7D
:10653000656D706F6F6C000061707000A465000085
:10654000000000206801000040040000F065000029
:1065500068010020E82B0000FC0A0000086500002C
:10656000000000001065000000000000146500003D
:10657000000000001C650000000000002465000011
:1065800000000003386500000000030394000020B1
:106590008C00002094000020A40400206001002052
:1065A00018000000017264200040542000400328BD
:1065B0007863326533A06433F86433A86433B86415
:1065C00033B06433C06433C86433D06433D86433C5
:1065D000E06433E86443F064041190D003C205061C
:1065E0004404192A3F4D333139031FF538000000A8
:0400000500000201F4
:00000001FF
